:02000000802E50
:03000B0002178D4C
:030023000202488E
:20002E000CB17581237508FF7509BF90A5ECE4F0123BF180EDC82581C822C92581C97A0079
:20004E0022D083D082CF2581F581CFC082C08322CF2581F581CF22FBE0CB22FCE0FBA3E06C
:20006E00CC22FAE0F9A3E0CA2229F9E5F03AFA227C00CB30E7011CCB2275F00030E70215FA
:20008E00F022FDE493A3FEE493A3FF4E7009E493FE740193FF800BE493A3B5050BE493B539
:2000AE00F0068F838E82E473A380D8FEEBA4FD8EF0ECA4FCEB8EF0A4C5F02C2DC5F0221131
:2000CE00D38EF0ED22C002C001AAF0F97E007D007F11C3E933F9EA33FADF08F5F0E9D0019C
:2000EE00D00222ED33FDEE33FEC3ED9BF5F0EE9C40E0ADF0FED380DBBB000122C333C5F096
:20010E0033C5F0DBF722BB000122C3C5F013C5F013DBF722240280022401C5F03400C5F065
:20012E0022C394028003C39401C5F09400C5F0223134F4C5F0F4C5F02245F0702204223144
:20014E00964024801A3196401E7014801A3196400E7014800A3196500E800431AA6008E4C7
:20016E00F5F02231AA60F8E4F5F0042231AA40F780ED31AA40F170E780ED31AA40E170E7A6
:20018E0080DD31AA50E180D7C39BC5F09C20E70720D207C345F02220D2F9D322C5F0C39CCD
:2001AE007003E5F09B2290A5ECE0A360EEE0FFA3E0A3CF2582F582EF3583F58380EB7E0040
:2001CE00CF2508F582EE3509F583EF227E00CF2508F9EE3509FAEF227E00C5082FC508C533
:2001EE00093EC50922E4F50AA88108E4F608B880FB22E4F520D201D200D203D205C2B4E4CB
:20020E00F50EF50DF50CF50BE4F512F511F510F50F74FFF513E588543FF588E589540FF512
:20022E00894420F5897450F598E5874480F58774FAF58BF58DD28ED2AC22C0E0C0D0C08365
:20024E00C082309839E50DB4FA028030502E050DE50DB50E0280044002F50E90A000C0E01B
:20026E00E50B2582F582E43583F583D0E0E599F0050BE50BB4FA004003750B00C29830999C
:20028E0048E511700DD200300235E4D5E0FDC2B4802DC20030011A300202D2B490A0FAC0F2
:2002AE00E0E5102582F582E43583F583D0E0E0F59915110510E510B4FA004003751000C2A3
:2002CE0099200105200002D299D082D083D0D0D0E0322278FB120043E6C0E0B40A0B300331
:2002EE0008D204740D1581C0E0E511B4FA0280F950F7C2AC90A0FAC0E0E50F2582F582E4C7
:20030E003583F583D0E0D0E0C0E0F00511050FE511B512004002F512E50FB4FA0040037525
:20032E000F00300002D299D2ACD0E0300408C204740AC0E080B322E4F5F078FB120043F6D9
:20034E0008A6F022E51364FF7038E50D6034300531C2AC90A000C0E0E50C2582F582E4357A
:20036E0083F583D0E0E0D2ACB40A0302038074018010150D050CE50CB4FA004003750C0085
:20038E0080C875F00022E4A20192E0F51F70030203B5E51160030203A0E4A20092E0F51F3C
:2003AE00E51F70030203A722C2AC7513FF7400F50CF50BC50DD2AC75F0002274FFC513B4AA
:2003CE00FF2EE50D0060FBC2AC90A000C0E0E50C2582F582E43583F583D0E0E0C0E0150DE2
:2003EE00050CE50CB4FA004003750C00D2ACD0E030050BB40A030203D0B40D02740A75F0D1
:20040E0000221203C9C0E0C0E0C0E01202E1D0E0D0E0D0E075F00022E51375F0007BFF7C0F
:20042E0000120169700302043E74FFF5F002044E78FB120043E60886F0F51318E60886F01F
:20044E002278FB1200438682088683E06016C083C082C0E0C0E01202E1D0E0D0E0D082D0F9
:20046E0083A380E722E4F5F078FB120043F608A6F022745D75F041C0E0C0F0E52075F00047
:20048E00C0E0C0F07402123D251581158115811581747875F041C0E0C0F0E50F75F000C0C1
:2004AE00E0C0F0E510C0E0C0F0E51175F000C0E0C0F0E512C0E0C0F0740575F000123D2515
:2004CE007FF612004F74AB75F041C0E0C0F0E50B75F000C0E0C0F0E50CC0E0C0F0E50D75D6
:2004EE00F000C0E0C0F0E50EC0E0C0F0740575F000123D257FF612004FE4F50EF512227FB4
:20050E00FD7EFF1201E8E4F5F07F001201CCF0A3C5F0F0C5F078FB120043E60886F0120105
:20052E003418F608A6F012012645F06022181818860108860289828A8312007089828A83CC
:20054E00E0120087C0E0C0F0123E1E1581158145F070030206197F001201CCE0A3F5F0E0BB
:20056E00C5F07B047C001201067F001201CCF0A3C5F0F0C5F078F9120043860108860289F3
:20058E00828A8312007089828A83E0120087C0E0C0F0123E2D158115817F021201CCF07FE3
:2005AE00021201CCE01200877B3912007E120153600B7F021201CCE0C39430800B7F0212D9
:2005CE0001CCE0C39441240A75F0007F001201CC1200692BC5F03CC5F07F001201CCF0A39A
:2005EE00C5F0F0C5F078F9120043860108860289828A83E0A3F5F0E0C5F012012689828AD3
:20060E0083F0A3C5F0F0C5F00205237F001201CCE0A3F5F0E0C5F07F030201E67FF17EFF7F
:20062E001201E87F021201DAE98AF0C0E0C0F0E4C0E0C0E0740A75F000C0E0C0F0123E5F8A
:20064E007FFA12004F7F021201DAE98AF07F0C1201CCF0A3C5F0F0C5F074097F0E1201CCA1
:20066E00F078FB120043860108860289828A8312007089828A83E0120087C0E0C0F0123DD3
:20068E00E51581158145F0602E78FB120043860108860289828A8312007089828A83E012F5
:2006AE000087C0E0C0F0123E191581158145F060067F0E1201CCE070030207397F0C120186
:2006CE00CCE0A3F5F0E0C5F01201267F0C1201CCF0A3C5F0F0C5F0120134F9AAF0C001C058
:2006EE000278F9120043860108860289828A8312007089828A83E0D083D082F0188601083F
:20070E00860289828A83E0A3F5F0E0C5F012012689828A83F0A3C5F0F0C5F07F0E1201CC84
:20072E00E0147F0E1201CCF002066F7F021201DAE98AF0C0E0C0F0123E82158115817F0046
:20074E001201CCF0A3C5F0F0C5F07F0F0201E67FFE7EFF1201E8E4F5F07F001201CCF0A399
:20076E00C5F0F0C5F07F001201CCE0A3F5F0E0C5F012014745F0601B78FB120043E6088670
:20078E00F012013418F608A6F01201267B007C0012015B45F0700302080378F7120043E66B
:2007AE000886F012012618F608A6F0120134F9AAF089828A83E0120087C0E0C0F008E60817
:2007CE0086F012012618F608A6F0120134F9AAF089828A83E0120087FBACF0D0F0D0E0C37B
:2007EE009BC5F09CC5F07F001201CCF0A3C5F0F0C5F00207737F001201CCE0A3F5F0E0C518
:20080E00F07F020201E67FFF7EFF1201E8E47F001201CCF07F001201CCE075F0007B107C9E
:20082E000012018070120208837F001201CCE0047F001201CCF080DC78FB120043E60886E0
:20084E00F07F001201CC1200652BC5F03400C5F0F9AAF07F001201CCE0C001C00279567A5F
:20086E00A412008712007789828A83E0F4D083D082F0020837740190A47AF07F010201E666
:20088E007FFF7EFF1201E8E4F521E4F5F090A2BEF0A3C5F0F0C5F0E490A2BDF074F475F024
:2008AE00A1C0E0C0F0E4C0E0C0E074C975F000C0E0C0F0123E5F7FFA12004FE4F5F090A39E
:2008CE0089F0A3C5F0F0C5F074C075F0A2C0E0C0F0E4C0E0C0E074C975F000C0E0C0F012E1
:2008EE003E5F7FFA12004FE490A455F0748C75F0A3C0E0C0F0E4C0E0C0E074C975F000C038
:20090E00E0C0F0123E5F7FFA12004F740190A47AF0E47F001201CCF07F001201CCE075F0C8
:20092E00007B107C0012017A70120209947F001201CCE0047F001201CCF080DC7F00120176
:20094E00CCE079567AA41200871200777F001201CCE0C001C00279687AA4120087120077EC
:20096E0089828A83E0F4120087D083D08212006512007E1201717003020991E490A47AF023
:20098E0002099402093B90A47AE060030209D9745675F0A4C0E0C0F0E4C0E0C0E07412754D
:2009AE00F000C0E0C0F0123E5F7FFA12004F745675F0A4C0E0C0F0745475F041C0E0C0F07F
:2009CE00123ECB15811581158115811236B31236B7746875F0A4C0E0C0F01208141581158E
:2009EE00817F010201E612039478FB120043E60886F090A38BF0C209C2B490A38BE075F038
:200A0E0000900A32020090E490A38BF0D208C202E490A522F0020A46C208D202E490A522E4
:200A2E00F0020A46260A0300260A0200260A01001A0A00000000150A227FFB7EFF1201E879
:200A4E0078F9120043E60886F07F031201CCF0A3C5F0F0C5F008E60886F07F011201CCF055
:200A6E00A3C5F0F0C5F07F011201DAE98AF0C0E0C0F0740275F000C0E0C0F012050D158166
:200A8E001581158115817F001201CCF078FB120043E60886F0C0E0C0F0743075F000C0E013
:200AAE00C0F07402C0E0C0F0123E5F7FFA12004F7F031201CC12007089828A83E0700302D9
:200ACE000B0A7F031201CC1200707F001201CCE089828A831200652B7F001201CCF07F0348
:200AEE001201CCE0A3F5F0E0C5F01201267F031201CCF0A3C5F0F0C5F0020ABE7F00120129
:200B0E00CCE0F4047F001201CCF078FB12004386010886027F001201CCE075F0007B047C58
:200B2E0000120114C001C00290415B12007012007789828A83E0D083D082F078FB12004371
:200B4E00E60886F02401C5F03400C5F0F9AAF07F001201CCE0540FC001C00290415B12006B
:200B6E007012008712007789828A83E0D083D082F07F001201CCE012008754FFC5F0540015
:200B8E00C5F07F050201E690A455E06003020C3B748C75F0A3C0E0C0F0E4C0E0C0E074C957
:200BAE0075F000C0E0C0F0123E5F7FFA12004F90A38BE075F0007B007C00120188700302DF
:200BCE000C27798C7AA3742489828A83F0E4A20992E0F51F748C75F0A3C0E0C0F0E51F6041
:200BEE000774EF75F041800574F375F041C0E0C0F0123EBB1581158115811581748C75F02D
:200C0E00A3C0E0C0F0745675F0A4C0E0C0F0123EBB1581158115811581748C75F0A3C0E0A5
:200C2E00C0F0123EF91581158190A455F078FB120043E60886F07B0A7C00120169700C18CB
:200C4E00E60886F07BFF7C0012016945F07003020CCCE4A20992E0F51F7003020C8F748C09
:200C6E0075F0A3C0E0C0F0748C75F0A32401C5F03400C0F0C0E0120A47158115811581156E
:200C8E0081748C75F0A3C0E0C0F012044F1581158178FB120043E60886F07B0A7C0012019C
:200CAE00697003020CC4740A75F000C0E0C0F01202E115811581E490A455F0020CF8748CC1
:200CCE0075F0A390A4551200652BC5F03400C5F0F9AAF078FB120043E60886F089828A835E
:200CEE00F090A455E00490A455F02278FB120043860108860289828A83E07003020D3A1843
:200D0E00860108860289828A83E0120087C0E0C0F0120B951581158178FB120043E60886B3
:200D2E00F012012618F608A6F0020CF9227FFA7EFF1201E8E4F5F07F021201CCF0A3C5F045
:200D4E00F0C5F078FB120043E60886F07F001201CCF0A3C5F0F0C5F0E47F041201CCF07FB4
:200D6E00041201CCE075F0007B027C0012017A7003020FBB7F041201CCE075F000900F91A1
:200D8E00020090C2097F001201CCE0A3F5F0E0C5F01201267F001201CCF0A3C5F0F0C5F009
:200DAE00120134F9AAF089828A83E0120087900F080200907F001201CC12007089828A8389
:200DCE00E01200877B2012007E1201697003020DEA74017F041201CCF0020DF274037F04B7
:200DEE001201CCF0020F1478FB120043E60886F0C0E0C0F018E60886F02401C5F03400C02B
:200E0E00F0C0E0120A4715811581158115817F051201CCF07F051201CCE07003020EA87444
:200E2E00037F041201CCF0742F75F075C0E0C0F090A2BEE0A3F5F0E0C5F012012690A2BE6C
:200E4E00F0A3C5F0F0C0F0C0E0123F40158115811581158190A2BEF0A3C5F0F0C5F090A303
:200E6E008BE075F0007B027C001201697003020EA574F575F041C0E0C0F07F051201CCE055
:200E8E0075F000C0E0C0F0740275F000123D251581158115811581020EFA7F001201CCE0A0
:200EAE00A3F5F0E0C5F02402C5F03400C5F07F001201CCF0A3C5F0F0C5F07F001201CC1288
:200ECE00007089828A83E01200877B2012007E1201697003020EF274017F041201CCF0D24E
:200EEE0009020EFA74037F041201CCF0020F1474037F041201CCF0020F14F50D2300C20D01
:200F0E0021000000FD0E020F9D745675F0A4C0E0C0F07F001201CCE0A3F5F0E0C0F0C0E0D0
:200F2E00745675F0A4C0E0C0F0123EF915811581C0E0C0F012075D7FFA12004F45F07003C3
:200F4E00020F5C74037F041201CCF0020F8E74027F041201CCF0745675F0A4C0E0C0F012B1
:200F6E003EF9158115817F001201CC1200692BC5F03CC5F07F021201CCF0A3C5F0F0C5F009
:200F8E00020F9D170F0100910D000000009D0F7F001201CCE0A3F5F0E0C5F01201267F0011
:200FAE001201CCF0A3C5F0F0C5F0020D6D7F021201CCE0A3F5F0E0C5F07F060201E67FFD94
:200FCE007EFF1201E8E4F5F07F011201CCF0A3C5F0F0C5F012035245F0700302126F1203CF
:200FEE00C97F001201CCF0E4A20892E0F51F70030210157F001201CCE0120087C0E0C0F0F7
:20100E001202E11581158190A2BDE0600302103D74F475F0A1C0E0C0F0E4C0E0C0E074C901
:20102E0075F000C0E0C0F0123E5F7FFA12004F7F001201CCE01200879010B502009090A274
:20104E00BDE0700302106E90A2BDE01490A2BDF079F47AA1120087120077E489828A83F09A
:20106E000210C10210C174F475F0A190A2BD1200652BC5F03400C5F0F9AAF07F001201CC2E
:20108E00E089828A83F090A2BDE00490A2BDF075F0007BC87C0012019070030210B274C76F
:2010AE0090A2BDF00210C171100A004C100800000074107F001201CCE01200877B0A12008F
:2010CE007E120169700302126F90A38BE075F00090125602009079F47AA189828A83E012F3
:2010EE0000877B2A12007E120171700302110E74F475F0A17F011201CCF0A3C5F0F0C5F054
:20110E0002126A74F475F0A1C0E0C0F0120D3B158115817F011201CCF0A3C5F0F0C5F002B1
:20112E00126A90A2BDE070030211AD79F47AA189828A83E012008790119D0200900211AD7A
:20114E00740C75F042C0E0C0F012044F1581158174F475F0A1C0E0C0F012044F158115812A
:20116E00740E75F042C0E0C0F012044F1581158174F475F0A1C0E0C0F0120D3B1581158113
:20118E007F011201CCF0A3C5F0F0C5F00211AD4B112D004B112A004B11240000004E110245
:2011AE00126A90A2BDE0700302124079F47AA189828A83E01200879012300200900212403E
:2011CE0074F475F0A1C0E0C0F0120D3B158115817F011201CCF0A3C5F0F0C5F07F011201DE
:2011EE00CCE0A3F5F0E0C5F045F0700302122D741075F042C0E0C0F012044F1581158174AF
:20120E005675F0A4C0E0C0F012044F15811581741475F042C0E0C0F012044F15811581026E
:20122E001240CB112D00CB112A00CB1124000000CE1102126A740175F000C0E0C0F012099D
:20124E00F41581158102126AB01103003011020011110100E410000000004312E490A2BD9C
:20126E00F07F011201CCE0A3F5F0E0C5F07F030201E690A38BE075F0007B007C0012016933
:20128E00700E90A38BE075F0007B027C0012016945F070030212B978FB120043E60886F0A9
:2012AE00C0E0C0F0120CF9158115812290A38BE075F0007B007C0012016970030212ED740D
:2012CE005675F0A4C0E0C0F012044F15811581741875F042C0E0C0F012044F15811581228A
:2012EE007FFD7EFF1201E878FB120043E60886F02401C5F03400C5F0F9AAF089828A83E072
:20130E001200877B3D12007E120169700302144918E60886F02402C5F03400C5F07F0012BF
:20132E0001CCF0A3C5F0F0C5F07F001201CCE0A3F5F0E0C0F0C0E0123EF9158115817B01FE
:20134E007C001201637003021436745675F0A4C0E0C0F0E4C0E0C0E0741275F000C0E0C03C
:20136E00F0123E5F7FFA12004FE47F021201CCF07F021201CCE075F0007B107C0012017A79
:20138E00600D7F001201CC12007089828A83E070120213F37F021201CCE0047F021201CCCC
:2013AE00F080CD7F021201CCE079567AA41200871200777F001201CCE0A3F5F0E0C5F01226
:2013CE0001267F001201CCF0A3C5F0F0C5F0120134C001C002F9AAF089828A83E0D083D015
:2013EE0082F00213A2745675F0A4C0E0C0F0745675F0A4C0E0C0F0123EF915811581D00427
:20140E00D0032BC5F03CC5F0F9AAF0742089828A83F01236B3746875F0A4C0E0C0F01208A1
:20142E001415811581021446741A75F042C0E0C0F0121280158115810214941236B374682C
:20144E0075F0A4C0E0C0F01208141581158174C075F0A2C0E0C0F0743475F042C0E0C0F0A1
:20146E00745675F0A4C0E0C0F0740375F000123D367FFA12004F74C075F0A2C0E0C0F01263
:20148E000CF9158115817F030201E678FB120043E60886F018F608A6F074C075F0A2C0E0EF
:2014AE00C0F0744775F042C0E0C0F0745675F0A4C0E0C0F0740375F000123D367FFA1200AD
:2014CE004F74C075F0A2C0E0C0F0120CF915811581788018E660FC881F74C075F0A2C0E00D
:2014EE00C0F0745875F042C0E0C0F0E51F75F000C0E0C0F0747FC0E0C0F0740475F0001280
:20150E003D367FF812004F74C075F0A2C0E0C0F0120CF9158115812278FB120043E6088646
:20152E00F018F608A6F074C075F0A2C0E0C0F0747275F042C0E0C0F0E50A75F000C0E0C0E5
:20154E00F090A2BEE0A3F5F0E0C0F0C0E0740475F000123D367FF812004F74C075F0A2C0D0
:20156E00E0C0F0120CF915811581E4F50AE4F5F090A2BEF0A3C5F0F0C5F0227FFE7EFF12D3
:20158E0001E878FB120043E60886F02401C5F03400C5F07F001201CCF0A3C5F0F0C5F07F9B
:2015AE00001201CC12007089828A83E0120087C0E0C0F0123E191581158145F07003021587
:2015CE00EB7F001201CCE0A3F5F0E0C0F0C0E0123E821581158190A522F002162574C075F1
:2015EE00F0A2C0E0C0F074A175F042C0E0C0F090A522E075F000C0E0C0F0740375F0001215
:20160E003D367FFA12004F74C075F0A2C0E0C0F0120CF9158115817F020201E67FFE7EFF3D
:20162E001201E878FB120043E60886F02401C5F03400C5F07F001201CCF0A3C5F0F0C5F067
:20164E007F001201CC12007089828A83E01200879016F902009074C075F0A2C0E0C0F074DB
:20166E00B575F042C0E0C0F090A38BE075F000C0E0C0F0740375F000123D367FFA12004F22
:20168E0074C075F0A2C0E0C0F0120CF9158115810217017F001201CC12007089828A83E07C
:2016AE00120087C0E0C0F0123E191581158145F070030216E67F001201CCE0A3F5F0E0C092
:2016CE00F0C0E0123E8215811581C0E0C0F01209F4158115810216F674C575F042C0E0C095
:2016EE00F012128015811581021701641600000000A1167F020201E690A38BE075F0007BE9
:20170E00007C00120169700302175574C075F0A2C0E0C0F074DD75F042C0E0C0F078F7128E
:20172E000043E60886F0C0E0C0F0740375F000123D367FFA12004F74C075F0A2C0E0C0F0DE
:20174E001212801581158122E4F522740F75F0EEF51485F015E4F516E4F517E4F518E4F57C
:20176E0019F51AE58854CFF588E58954F0F5894401F589E4F58AF58CD2B9D2A9D28C22C009
:20178E00E0C0D0C28C85148A85158CD28CC0F0C083C082C00020164675F0FF109702C2F79F
:2017AE00109602C2F6109502C2F5109402C2F4109302C2F3109202C2F2109102C2F1109059
:2017CE0002C2F085F0904390F0E59085F090F454F0F5F0651985F019600455F0421AE518DA
:2017EE006007C294D5E002D294F51805170516E516B4C8004006D2172438F516D000D0828E
:20180E00D083D0F0D0D0D0E032227FFF7EFF1201E8E5167F001201CCF07F001201CCE07511
:20182E00F000AB167C00120169600302182778FB120043E60886F012013418F608A6F0121C
:20184E00012645F0600302181F7F010201E678FB120043E60886F045F0700302188A75F03C
:20186E002ED5F0FD78FB120043E60886F012013418F608A6F045F0600302186C2278FB1286
:20188E000043E60886F0C0E0C0F0120CF91581158174F875F042C0E0C0F0120CF9158115DB
:2018AE008112035245F070030218AF74FF75F042C0E0C0F0120CF9158115810203C97FFEC9
:2018CE007EFF1201E8E4F5F07F001201CCF0A3C5F0F0C5F0E4A21F92E0F51F600302198045
:2018EE00E4F517B297E4C0E0C0E0121991158115817F001201CCF0A3C5F0F0C5F0B2977F82
:20190E00001201CCE0A3F5F0E0C5F05480C5F05400C5F045F0600690A522E05402700302AE
:20192E001940747775F000C0E0C0F0120B9515811581E51775F0007B0A7C00120188700352
:20194E00021965D21FE4F5F07F001201CCF0A3C5F0F0C5F00219807F001201CCE0A3F5F093
:20196E00E0C5F05480C5F05400C5F045F060030218F17F001201CCE0A3F5F0E0C5F07F02B3
:20198E000201E67FFF7EFF1201E8D216E590440FF59078FB120043E60886F07B017C0012EF
:2019AE00016970030219BAD2B50219BCC2B5D2B2D2B3E590540F7F001201CCF07F001201D1
:2019CE00CCE075F0007B047C001201067F001201CCF0C2B3D2B3E590540F7F001201CC1244
:2019EE0000654B7F001201CCF0C2B3C2167F001201CCE075F0007F010201E67FFF7EFF1275
:201A0E0001E878FB120043E60886F05402C5F05400C5F045F06003021A2B1218CCD216785A
:201A2E00FB120043E60886F05401C5F05400C5F045F07003021A4AD2B5021A4CC2B5C2B2E9
:201A4E00E59054F0120087C0E0C0F078F7120043E60886F07B047C00120114540FC5F05420
:201A6E00FFC5F0D004D0034BC5F04CC5F07F001201CCF07F001201CCE0F590D2B3C2B3E50C
:201A8E009054F0120087C0E0C0F018E60886F0540FC5F054FFC5F0D004D0034BC5F04CC527
:201AAE00F07F001201CCF07F001201CCE0F590D2B3C2B3D2B2C2167F010201E690A522E021
:201ACE0054027003021AE5740175F043C0E0C0F0120CF915811581E4F523E4F51DF51C90EB
:201AEE00414AE0F51BE590440FF590C2B3C2B5C2B2D216740375F000C0E0C0F01218181545
:201B0E00811581E59054F04403F590D2B3C2B3740175F000C0E0C0F012181815811581E5A4
:201B2E009054F04403F590D2B3C2B3740275F000C0E0C0F012185C15811581E59054F04423
:201B4E0003F590D2B3C2B3740175F000C0E0C0F012181815811581E59054F04402F590D207
:201B6E00B3C2B3C216742875F000C0E0C0F0E4C0E0C0F0121A0915811581158115817408C9
:201B8E0075F000C0E0C0F0E4C0E0C0F0121A091581158115811581740175F000C0E0C0F097
:201BAE00E4C0E0C0F0121A091581158115811581740675F000C0E0C0F0E4C0E0C0F0121AC7
:201BCE0009158115811581158190414BE0440CF51E75F000C0E0C0F0E4C0E0C0E0121A0929
:201BEE00158115811581158190A522E054027003021C11741975F043C0E0C0F0120CF9159F
:201C0E00811581227FFF7EFF1201E878F9120043E60886F0C0E0C0F0E4C0E0C0E0123F2474
:201C2E00158115811581158178F9120043F608A6F008E60886F0C0E0C0F0E4C0E0C0E012F2
:201C4E003F24158115811581158178FB120043F608A6F0181818E60886F0C0E0C0F0904192
:201C6E0048E0C3940175F000C0E0C0F0123F40158115811581158178F9120043F608A6F0DE
:201C8E00F51C08E60886F0C0E0C0F0904149E0C3940175F000C0E0C0F0123F4015811581A5
:201CAE001581158178FB120043F608A6F0F51D181818E60886F0794C7A4112007789828A32
:201CCE0083E075F00078FB12004326C5F00836C5F04480C5F04400C5F07F001201CCF09048
:201CEE00A522E054027003021D4874C075F0A2C0E0C0F0742075F043C0E0C0F0181818E6BA
:201D0E000886F0C0E0C0F008E60886F0C0E0C0F07F001201CCE075F000C0E0C0F07405754A
:201D2E00F000123D367FF612004F74C075F0A2C0E0C0F0120CF9158115817F001201CCE03E
:201D4E0075F000C0E0C0F0E4C0E0C0E0121A0915811581158115817F010201E6E4F51DF5BB
:201D6E001C740275F000C0E0C0F0E4C0E0C0F0121A09158115811581158122E4F51DF51C24
:201D8E00740175F000C0E0C0F0E4C0E0C0F0121A091581158115811581227FFB7EFF12011E
:201DAE00E890A522E054027003021DF674C075F0A2C0E0C0F0743E75F043C0E0C0F078F774
:201DCE00120043E60886F0C0E0C0F0740375F000123D367FFA12004F74C075F0A2C0E0C016
:201DEE00F0120CF91581158178FB120043E60886F045F0700302204B78FB120043E6088625
:201E0E00F09041481200657C001201907003021E25121D8902204BE51B20E103021E39E4F7
:201E2E00C0E0C0E0122094158115811218CCE51C7F001201CCF0E51D7F011201CCF078FB59
:201E4E00120043E60886F07F021201CCF0E47F031201CCF07F021201CCE075F00090414878
:201E6E001200657C0012017A701F021F917F021201CCE0047F021201CCF07F031201CCE0BE
:201E8E00047F031201CCF080CB7F021201CCE075F000C0E0C0F0E4C0E0C0E0121C121581A5
:201EAE00158115811581E47F041201CCF07F041201CCE075F0009041491200657C00120155
:201ECE007A7012021F0F7F041201CCE0047F041201CCF080D87F041201CCE0797B7AA4750F
:201EEE00F000120077C001C002740175F000C0E0C0F012199115811581D083D082F0021E11
:201F0E00D47F031201CCE075F000C0E0C0F0E4C0E0C0E0121C121581158115811581E47FCA
:201F2E00041201CCF07F041201CCE075F0009041491200657C0012017A7012021F8E7F04CB
:201F4E001201CCE0047F041201CCF080D87F041201CCE0797B7AA475F00012007789828A2F
:201F6E0083E075F000C0E0C0F0740175F000C0E0C0F0121A091581158115811581021F4C17
:201F8E00021E7B904148E0C3940175F000C0E0C0F0E4C0E0C0E0121C121581158115811557
:201FAE0081E47F041201CCF07F041201CCE075F0009041491200657C0012017A7012021F78
:201FCE00FB7F041201CCE0047F041201CCF080D8742075F000C0E0C0F07401C0E0C0F012E8
:201FEE001A091581158115811581021FCF7F001201CCE075F000C0E0C0F07F011201CCE036
:20200E0075F000C0E0C0F0121C121581158115811581740175F000C0E0C0F01220941581DF
:20202E00158190A522E05402700302204B745475F043C0E0C0F0120CF9158115817F050206
:20204E0001E678FB120043E60886F090206E020090E4F51E02207A90414BE0F51E02207A71
:20206E00652001005F20000000007A20E51E75F000C0E0C0F0E4C0E0C0F0121A09158115E7
:20208E008115811581227FFE7EFF1201E8E51E440875F0007F001201CCF0A3C5F0F0C5F06F
:2020AE0078FB120043E60886F07B017C001201696007740475F0008003E4F5F07F00120150
:2020CE00CC1200694BC5F04CC5F07F001201CCF0A3C5F0F0C5F07F001201CCE0A3F5F0E0B9
:2020EE00C0F0C0E0E4C0E0C0E0121A0915811581158115817F020201E67FFE7EFF1201E872
:20210E0090A522E05402700302217C74C075F0A2C0E0C0F0746575F043C0E0C0F078F71235
:20212E000043E6120087C0E0C0F0E6120087C0E0C0F0123E121581158145F06007742D7570
:20214E00F000800678F5120043E6120087C0E0C0F0740475F000123D367FF812004F74C0FC
:20216E0075F0A2C0E0C0F0120CF91581158178FB120043E61200879024BB02009090414856
:20218E00E0C3940175F000AB1C7C0012016970030221C2E51B20E0030221BC740175F000C1
:2021AE00C0E0C0F0121DA8158115810221BFE4F51C0221C6051CE51CE51B30E2030221EBB9
:2021CE00E51C75F000C0E0C0F0E51DC0E0C0F0121C1215811581158115810224D3E51C75E2
:2021EE00F000C0E0C0F0E4C0E0C0F0121C1215811581158115810224D3121D890224D3E536
:20220E001D7003022218151DE51DE51B20E4030224D31218CCE51B20E103022237E4C0E0D7
:20222E00C0E01220941581158190A522E054027003022252747475F043C0E0C0F0120CF991
:20224E0015811581E51D7F001201CCF07F001201CCE075F0009041491200657C00120180B1
:20226E0070120222EF7F001201CCE0047F001201CCF080D87F001201CCE0797B7AA475F01E
:20228E0000120077C001C002740175F000C0E0C0F012199115811581D083D082F07F0112EB
:2022AE0001CCF090A522E0540270030222EC7F011201CCE075F000C0E0C0F0123E0D15815C
:2022CE00158145F060087F011201CCE08005742D75F000C0E0C0F0120B95158115810222A1
:2022EE007390A522E05402700302230A748B75F043C0E0C0F0120CF915811581E51C75F08E
:20230E0000C0E0C0F0E51DC0E0C0F0121C12158115811581158190A522E054027003022350
:20232E003F748E75F043C0E0C0F0120CF915811581E51D24017F001201CCF07F001201CC40
:20234E00E075F0009041491200657C0012017A70120223EB7F001201CCE0047F001201CC5E
:20236E00F080D87F001201CCE0797B7AA475F00012007789828A83E07F011201CCF07F0102
:20238E001201CCE075F000C0E0C0F0740175F000C0E0C0F0121A0915811581158115819074
:2023AE00A522E0540270030223E87F011201CCE075F000C0E0C0F0123E0D1581158145F0E0
:2023CE0060087F011201CCE08005742D75F000C0E0C0F0120B9515811581022362742075FF
:2023EE00F000C0E0C0F07401C0E0C0F0121A09158115811581158190A522E054027003023B
:20240E00242074A575F043C0E0C0F0120CF915811581E51C75F000C0E0C0F0E51DC0E0C0FE
:20242E00F0121C121581158115811581740175F000C0E0C0F0122094158115810224D37879
:20244E00FB120043E6120087C0E0C0F0740175F000C0E0C0F0121A09158115811581158198
:20246E00051DE51DE51D75F0009041491200657C0012019070030224B8E51C75F000C0E0BC
:20248E00C0F0E4C0E0C0F0121C121581158115811581E51B30E3030224B8740A75F000C01B
:2024AE00E0C0F0122107158115810224D320227F000D22080007220C00EB210D008B210A23
:2024CE000000004D247F020201E678FB120043860108860289828A83E01200877B00120016
:2024EE007E120171700302252418860108860289828A83E0120087C0E0C0F012210715812E
:20250E00158178FB120043E60886F012012618F608A6F00224D822740190A4CCF0E490A469
:20252E00CFF090A4CEF0740190A521F090A520F02290A522E0540170030225B974C075F042
:20254E00A2C0E0C0F074A975F043C0E0C0F078F7120043E60886F0C0E0C0F018E60886F072
:20256E00C0E0C0F0123E0D1581158145F0600B78F5120043E60886F08005742D75F000C063
:20258E00E0C0F090A4CCE075F000C0E0C0F0740575F000123D367FF612004F74C075F0A294
:2025AE00C0E0C0F0120CF91581158190A4CCE075F0007B007C0012016970030225E378FBD2
:2025CE00120043E60886F0C0E0C0F01221071581158102291590A4CEE079D07AA475F00090
:2025EE0012007778FB120043E60886F0547FC5F05400C5F089828A83F090A4CEE00490A465
:20260E00CEF075F000C0E0C0F0743F75F000C0E0C0F0123F40158115811581158190A4CEE6
:20262E00F090A4CCE075F000902901020090E490A4CFF090A4CEF078FB120043E60886F016
:20264E007B1B7C00120169700302269D90A522E05401700302267574CF75F043C0E0C0F0CF
:20266E00120CF91581158174D075F0A4C0E0C0F0E4C0E0C0E0744075F000C0E0C0F0123E8F
:20268E005F7FFA12004F740290A4CCF00226B178FB120043E60886F0C0E0C0F012210715E9
:2026AE0081158102291578FB120043E60886F07B5B7C0012016970030226D2740390A4CCD7
:2026CE00F002270190A522E0540170030226ED74E775F043C0E0C0F0120CF91581158178B0
:2026EE00FB120043E60886F0C0E0C0F0122B561581158102291578FB120043E60886F07B22
:20270E003D7C001201697003022722740390A4CCF00227FE78FB120043E60886F0C0E0C09E
:20272E00F0123E191581158145F07003022746740490A4CCF00227FE78FB120043E6088624
:20274E00F0C0E0C0F0123DFE1581158145F0700302277B12291678FB120043E60886F0C029
:20276E00E0C0F0122BD0158115810227FE90A522E0540170030227EA74C075F0A2C0E0C0AE
:20278E00F0740F75F044C0E0C0F078F7120043E60886F0C0E0C0F018E60886F0C0E0C0F07B
:2027AE00123E0D1581158145F0600B78F5120043E60886F08005742D75F000C0E0C0F0746D
:2027CE000475F000123D367FF812004F74C075F0A2C0E0C0F0120CF91581158178FB1200D2
:2027EE0043E60886F0C0E0C0F0122B561581158102291578FB120043E60886F07B3B7C0077
:20280E00120169700302281C1229160228F878FB120043E60886F0C0E0C0F0123E19158187
:20282E00158145F07003022840740490A4CCF00228F878FB120043E60886F0C0E0C0F012CA
:20284E003DFE1581158145F0700302287512291678FB120043E60886F0C0E0C0F0122BD0E2
:20286E00158115810228F890A522E0540170030228E474C075F0A2C0E0C0F0743275F04415
:20288E00C0E0C0F078F7120043E60886F0C0E0C0F018E60886F0C0E0C0F0123E0D1581158E
:2028AE008145F0600B78F5120043E60886F08005742D75F000C0E0C0F0740475F000123DBC
:2028CE00367FF812004F74C075F0A2C0E0C0F0120CF91581158178FB120043E60886F0C022
:2028EE00E0C0F0122B56158115810229151225250229150128040004270300B42602003C2C
:20290E002601000000FB28227FFC7EFF1201E890A522E05401700302296E74C075F0A2C0B7
:20292E00E0C0F0746175F044C0E0C0F074D075F0A4C0E0C0F090A4CEE0C3940275F000C02E
:20294E00E0C0F0740475F000123D367FF812004F74C075F0A2C0E0C0F0120CF915811581D1
:20296E0074D075F0A490A4CE1200652BC5F03400C5F0C39402C5F09400C5F07F021201CC03
:20298E00F0A3C5F0F0C5F074D075F0A47F021201CC1200691201807020022A527F021201DF
:2029AE00CCE0A3F5F0E0C5F01201347F021201CCF0A3C5F0F0C5F080CE7F021201CC1200EC
:2029CE007089828A83E0120087C0E0C0F0123E191581158145F06003022A4F7F021201CC90
:2029EE00E0A3F5F0E0C5F01201267F021201CCF0A3C5F0F0C5F090A522E054017003022A1B
:202A0E004C74C075F0A2C0E0C0F0748675F044C0E0C0F07F021201CCE0A3F5F0E0C0F0C0C6
:202A2E00E0740375F000123D367FFA12004F74C075F0A2C0E0C0F0120CF915811581022A73
:202A4E00520229AA7F021201CC12007089828A83E0120087C0E0C0F0123E191581158145A4
:202A6E00F07003022A987F021201CCE0A3F5F0E0C0F0C0E0123E82158115817F001201CCCD
:202A8E00F0A3C5F0F0C5F0022AA9740175F0007F001201CCF0A3C5F0F0C5F090A4CFE075E9
:202AAE00F000C333C5F033C5F079107AA51200777F001201CCE0A3F5F0E0C5F089828A83E1
:202ACE00F0A3C5F0F0C5F090A4CFE00490A4CFF075F000C0E0C0F0740775F000C0E0C0F03C
:202AEE00123F40158115811581158190A4CFF090A522E054017003022B4574C075F0A2C080
:202B0E00E0C0F0749D75F044C0E0C0F07F001201CCE0A3F5F0E0C0F0C0E0740375F0001229
:202B2E003D367FFA12004F74C075F0A2C0E0C0F0120CF9158115817F001201CCE0A3F5F0A6
:202B4E00E0C5F07F040201E678FB120043E60886F018F608A6F090A4CEE07003022BC090BC
:202B6E00A522E054017003022BA074C075F0A2C0E0C0F074A275F044C0E0C0F074D075F0C8
:202B8E00A4C0E0C0F0740375F000123D367FFA12004F741B75F000C0E0C0F01221071581E4
:202BAE00158174D075F0A4C0E0C0F01224D815811581E490A4CFF090A4CEF0740190A4CC5C
:202BCE00F0227FFF7EFF1201E890A522E054017003022BF274BC75F044C0E0C0F0120CF981
:202BEE0015811581740190A4CCF078FB120043E60886F090324702009090A522E054017073
:202C0E0003022C5874C075F0A2C0E0C0F074CF75F044C0E0C0F0E4F5F079107AA51200775C
:202C2E0089828A83E0A3F5F0E0C0F0C0E0740375F000123D367FFA12004F74C075F0A2C0A0
:202C4E00E0C0F0120CF915811581E4F5F079107AA5120077E51C75F00089828A83120069A0
:202C6E00C39BC5F09CC0F0C0E0E51D75F000C0E0C0F0121C12158115811581158102328F35
:202C8E0090A522E054017003022CDF74C075F0A2C0E0C0F074E075F044C0E0C0F0E4F5F079
:202CAE0079107AA512007789828A83E0A3F5F0E0C0F0C0E0740375F000123D367FFA120039
:202CCE004F74C075F0A2C0E0C0F0120CF915811581E4F5F079107AA5120077E51C75F00069
:202CEE0089828A831200692BC5F03CC0F0C0E0E51D75F000C0E0C0F0121C1215811581158F
:202D0E0081158102328F90A522E054017003022D6574C075F0A2C0E0C0F074F375F044C0DD
:202D2E00E0C0F0E4F5F079107AA512007789828A83E0A3F5F0E0C0F0C0E0740375F000125D
:202D4E003D367FFA12004F74C075F0A2C0E0C0F0120CF915811581E51C75F000C0E0C0F094
:202D6E00E479107AA5120077E51D75F00089828A831200692BC5F03CC0F0C0E0121C121575
:202D8E008115811581158102328F90A522E054017003022DE974C075F0A2C0E0C0F0740900
:202DAE0075F045C0E0C0F0E4F5F079107AA512007789828A83E0A3F5F0E0C0F0C0E07403EA
:202DCE0075F000123D367FFA12004F74C075F0A2C0E0C0F0120CF915811581E51C75F000ED
:202DEE00C0E0C0F0E479107AA5120077E51D75F00089828A83120069C39BC5F09CC0F0C047
:202E0E00E0121C12158115811581158102328F90A4CFE075F0007B027C0012017A700E021B
:202E2E002E6390A4CFE00490A4CFF080E290A4CFE075F000C333C5F033C5F079107AA51222
:202E4E000077740175F00089828A83F0A3C5F0F0C5F0022E3090A522E054017003022ECDB2
:202E6E0074C075F0A2C0E0C0F0741C75F045C0E0C0F0E4F5F079107AA512007789828A831D
:202E8E00E0A3F5F0E0C0F0C0E0740275F00079107AA512007789828A83E0A3F5F0E0C0F070
:202EAE00C0E0740475F000123D367FF812004F74C075F0A2C0E0C0F0120CF915811581E478
:202ECE00F5F079107AA512007789828A83E0A3F5F0E0C5F0C39401C5F09400C0F0C0E07454
:202EEE000275F00079107AA512007789828A83E0A3F5F0E0C5F0C39401C5F09400C0F0C006
:202F0E00E0121C12158115811581158102328FE4F5F079107AA512007789828A83E0A3F5DE
:202F2E00F0E0C5F07B027C001201697003022F5C90A522E054017003022F59743E75F045A4
:202F4E00C0E0C0F0120CF915811581121D8902328F90A522E054017003022F7A745775F07B
:202F6E0045C0E0C0F0120CF915811581904149E0C3951D7F001201CCF07F001201CCE07000
:202F8E0003022FB2747F75F000C0E0C0F0122107158115817F001201CCE0147F001201CC7F
:202FAE00F0022F8702328F02328FE4F5F079107AA512007789828A83E0A3F5F0E0C5F07B4B
:202FCE00077C001201697003022FFA90A522E054017003022FF4746F75F045C0E0C0F01233
:202FEE000CF915811581E51B4408F51B02328FE4F5F079107AA512007789828A83E0A3F5E9
:20300E00F0E0C5F07B077C00120169700302303F90A522E054017003023039748575F045B2
:20302E00C0E0C0F0120CF915811581E51B54F7F51B02328F02328F90A522E054017003020D
:20304E00309574C075F0A2C0E0C0F0749D75F045C0E0C0F0E51C240175F000C0E0C0F0E547
:20306E001D240175F000C0E0C0F0740475F000123D367FF812004F74C075F0A2C0E0C0F086
:20308E00120CF91581158174C075F0A2C0E0C0F074C775F045C0E0C0F0E51C240175F00094
:2030AE00C0E0C0F0E51D240175F000C0E0C0F0740475F000123D367FF812004F74C075F003
:2030CE00A2C0E0C0F0120CF91581158102328F02328FE51C240190A520F0E51D240190A560
:2030EE0021F090A522E05401700302314074C075F0A2C0E0C0F074D175F045C0E0C0F090E5
:20310E00A520E075F000C0E0C0F090A521E075F000C0E0C0F0740475F000123D367FF81271
:20312E00004F74C075F0A2C0E0C0F0120CF91581158102328F90A522E054017003023193DC
:20314E0074C075F0A2C0E0C0F074F675F045C0E0C0F090A520E075F000C0E0C0F090A52132
:20316E00E075F000C0E0C0F0740475F000123D367FF812004F74C075F0A2C0E0C0F0120CC9
:20318E00F91581158190A520E0C3940175F000C0E0C0F090A521E0C3940175F000C0E0C067
:2031AE00F0121C12158115811581158102328F90A522E05401700302323074C075F0A2C058
:2031CE00E0C0F0741E75F046C0E0C0F078F7120043E60886F0C0E0C0F0123E1215811581BE
:2031EE0045F0600B78F7120043E60886F08005742D75F000C0E0C0F078F5120043E60886E8
:20320E00F0C0E0C0F0740475F000123D367FF812004F74C075F0A2C0E0C0F0120CF91581EE
:20322E00158178FB120043E60886F0C0E0C0F0122B561581158102328F43317500E0307380
:20324E0000DD30700045306E0042306D00FD2F6C00B82F6800B52F52005F2F4B001D2F4A95
:20326E00001D2E6A001D2E66001D2E4800982D4400142D43008E2C4200072C41000000BD8D
:20328E003190A522E0540170030232AA744475F046C0E0C0F0120CF9158115817F01020199
:2032AE00E67FED7EFF1201E878FB120043860108860289828A83E070030236AE188601085F
:2032CE00860289828A83E01200877B5C12007E120169700302367D18E60886F02401C5F066
:2032EE003400C5F0F9AAF089828A83E0120087C0E0C0F0123E46158115819035DD0200906D
:20330E00E4F5F07F001201DA120077E489828A83F07464F518023605E4F5F07F001201DA9E
:20332E0012007778FB120043E60886F02402C5F03400C5F0C001C002F9AAF089828A83E0F8
:20334E00541FD083D082F0740175F0007F001201DA120077E489828A83F078FB120043E6EE
:20336E000886F02401C5F03400C5F018F608A6F00236057F001201DAE98AF0C0E0C0F07482
:20338E004675F046C0E0C0F0123ECB15811581158115810236057F001201DAE98AF0C0E0BF
:2033AE00C0F0744875F046C0E0C0F0123ECB15811581158115810236057F001201DAE98A09
:2033CE00F0C0E0C0F0744A75F046C0E0C0F0123ECB15811581158115810236057F001201A4
:2033EE00DAE98AF0C0E0C0F0744C75F046C0E0C0F0123ECB1581158115811581023605E5E2
:20340E001D240175F0007B047C001200CDFB7404C39B7F0E1201CCF07F001201DAE98AF021
:20342E00C0E0C0F0742075F000C0E0C0F07F0E1201CCE075F000C0E0C0F0123E5F7FFA12AA
:20344E00004F7F0E1201CCE07F001201DA120087120077E489828A83F0023605E51C7F0F7D
:20346E001201CCF0E51D7F101201CCF0744E75F046C0E0C0F012253F15811581E51C7F111F
:20348E001201CCF0E51D7F121201CCF078FB120043E60886F02402C5F03400C5F07F0C1260
:2034AE0001CCF0A3C5F0F0C5F07F0C1201DAE98AF0C0E0C0F0740275F000C0E0C0F01205D7
:2034CE000D15811581158115817F0E1201CCF07F0F1201CCE075F000C0E0C0F07F10120179
:2034EE00CCE075F000C0E0C0F0121C1215811581158115817F0E1201CCE075F000C0E0C0B4
:20350E00F0740175F000C0E0C0F0121A0915811581158115817F111201CCE075F000C0E0A2
:20352E00C0F07F121201CCE075F000C0E0C0F0121C121581158115811581E4F5F07F0012D6
:20354E0001DA120077E489828A83F078FB120043E60886F02402C5F03400C5F018F608A661
:20356E00F0023605E4F5F07F001201DA120077745C89828A83F0740175F0007F001201DA34
:20358E00120077E489828A83F0023605E4F5F07F001201DA12007778FB120043E60886F081
:2035AE002401C5F03400C5F0C001C002F9AAF089828A83E0D083D082F0740175F0007F003E
:2035CE001201DA120077E489828A83F002360572355C006A3478000D347400EA337200C71A
:2035EE00336E00A433660081336500263363000E33620000009A3578FB120043E60886F06C
:20360E002402C5F03400C5F018F608A6F07F001201DAE98AF07F0A1201CCF0A3C5F0F0C5F8
:20362E00F07F0A1201CC12007089828A83E0700302367A7F0A1201CC12007089828A83E0A3
:20364E00120087C0E0C0F012253F158115817F0A1201CCE0A3F5F0E0C5F01201267F0A1298
:20366E0001CCF0A3C5F0F0C5F002362F0236AB78FB120043860108860289828A83E012004F
:20368E0087C0E0C0F012253F1581158178FB120043E60886F012012618F608A6F00232B6A8
:2036AE007F130201E6E4F5F022D294A294B3E492E0F51FE51F70030236D7E4C0E0C0E01221
:2036CE0009F4158115810236E7740175F000C0E0C0F01209F415811581227FFA7EFF120104
:2036EE00E8742375F0A5C0E0C0F074F475F0A1C0E0C0F0123ECB158115811581158178FB3F
:20370E00120043E60886F07F021201CCF0A3C5F0F0C5F07F001201CCF0A3C5F0F0C5F07FCB
:20372E00001201CC12007089828A83E070030237DF7F001201CC12007089828A83E01200AD
:20374E00877B2012007E120169700302377A7F001201CCE0A3F5F0E0C5F01201267F0012E2
:20376E0001CCF0A3C5F0F0C5F00237DC7F021201CC120070C001C0027F001201CC12007027
:20378E0089828A83E0120087C0E0C0F0123E2D15811581D083D082F07F001201CCE0A3F526
:2037AE00F0E0C5F01201267F001201CCF0A3C5F0F0C5F07F021201CCE0A3F5F0E0C5F01283
:2037CE0001267F021201CCF0A3C5F0F0C5F002372D7F021201CC120070E489828A83F078BB
:2037EE00FB120043E60886F02401C5F03400C5F07F001201CCF0A3C5F0F0C5F01886010852
:20380E00860289828A83E0120087903BBC02009078FB120043E60886F0C0E0C0F01212EEDA
:20382E0015811581023BEC121499023BEC78FB120043E60886F0C0E0C0F0121526158115C9
:20384E0081023BEC78FB120043E60886F0C0E0C0F012158915811581023BEC78FB12004367
:20386E00E60886F0C0E0C0F012162A15811581023BEC7F001201CCE0A3F5F0E0C5F024025E
:20388E00C5F03400C5F0F9AAF089828A83E0120087C39430C5F09400C5F07F041201CCF081
:2038AE00A3C5F0F0C5F07F001201CCE0A3F5F0E0C5F02401C5F03400C5F0F9AAF089828AB7
:2038CE0083E01200877B3D12007E12016960287F041201CCE0A3F5F0E0C5F07B007C00122A
:2038EE00016360137F041201CCE0A3F5F0E0C5F07B017C0012015345F0700302399F7F0025
:20390E001201CC12007089828A83E012008790398C0200907F041201CCE0A3F5F0E0C5F061
:20392E0045F0700302393AD29602393CC29602399C7F041201CCE0A3F5F0E0C5F045F0704A
:20394E0003023957D295023959C29502399C7F041201CCE0A3F5F0E0C5F045F07003023959
:20396E0074D294023976C29402399C745075F046C0E0C0F01212801581158102399C5C3986
:20398E0043003F39420022394100000079390239AF746975F046C0E0C0F0121280158115BD
:2039AE0081023BECD21674C075F0A2C0E0C0F0748275F046C0E0C0F0E51A75F000C0E0C027
:2039CE00F07403123D367FFA12004FE4F51AC21674C075F0A2C0E0C0F0120CF9158115817A
:2039EE00023BEC7F001201CCE0A3F5F0E0C0F0C0E0748875F046C0E0C0F0123F8715811520
:203A0E00811581158145F07003023A2D748D75F046C0E0C0F012128015811581023A33128D
:203A2E000394020000023BEC742375F0A5C0E0C0F0743D75F000C0E0C0F0123FBD158115A6
:203A4E0081158115817F001201CCF0A3C5F0F0C5F07F001201CCE0A3F5F0E0C5F045F06070
:203A6E00367F001201CC12007089828A83E01200877B3D12007E120169601C7F001201CCF3
:203A8E00E0A3F5F0E0C0F0C0E0123EF9158115817B017C0012015B45F07003023ACC7F0076
:203AAE001201CCE0A3F5F0E0C5F02401C5F03400C0F0C0E01232AF15811581023ADC74A271
:203ACE0075F046C0E0C0F012128015811581023BEC023BEC74C375F046C0E0C0F0120CF972
:203AEE001581158174F775F046C0E0C0F0120CF915811581742475F047C0E0C0F0120CF938
:203B0E0015811581746075F047C0E0C0F0120CF915811581748A75F047C0E0C0F0120CF947
:203B2E001581158174B375F047C0E0C0F0120CF91581158174D375F047C0E0C0F0120CF98B
:203B4E001581158174FE75F047C0E0C0F0120CF915811581742075F048C0E0C0F0120CF9D2
:203B6E0015811581745575F048C0E0C0F0120CF915811581748975F048C0E0C0F0120CF9F1
:203B8E001581158174A875F048C0E0C0F0120CF915811581023BEC78FB120043E60886F03A
:203BAE00C0E0C0F012170615811581023BECE23A3F00DF3A0000363A5300F1395200B23985
:203BCE00510080384F0069384E0052384C003B384500353844001E3841000000A53B7F0655
:203BEE000201E67FFD7EFF1201E81201F3121756120200D2AF12088E121ACA12252590A393
:203C0E008BE06003023C4574C475F048C0E0C0F0120CF91581158174EF75F048C0E0C0F06D
:203C2E00120CF91581158174F475F048C0E0C0F0120CF91581158174C075F0A2C0E0C0F000
:203C4E00741C75F049C0E0C0F0742A75F049C0E0C0F0740375F000123D367FFA12004F747D
:203C6E00C075F0A2C0E0C0F01232AF15811581742F75F049C0E0C0F01232AF15811581122E
:203C8E0012BAE47F021201CCF0740175F00045F07003023D10E4A21792E0F51F7003023C71
:203CAE00B7B297B297B297C217120FCC7F001201CCF0A3C5F0F0C5F07B007C001201717068
:203CCE0003023D0D7F021201CCE06003023CF5744475F049C0E0C0F01232AF158115817468
:203CEE00017F021201CCF07F001201CCE0A3F5F0E0C0F0C0E01236E8158115811212BA0233
:203D0E003C97744975F049C0E0C0F0120CF9158115817F030201E623F42581F81201B412CB
:203D2E003FDA1201B402045923F42581F8868208868308023FDA0000000000000000002025
:203D4E0020202020000000000000000000000000000000000000600101010101010101016C
:203D6E0001010101010118181818181818181818010101010101010A0A0A0A0A0A020202F6
:203D8E0002020202020202020202020202020202020101010101010C0C0C0C0C0C04040499
:203DAE0004040404040404040404040404040404040101010100C2D578FB120043E6903D9B
:203DCE0044C2E79355F060027401A2D575F00092F065F075F0002278FB120043E6A2E7B315
:203DEE00E4F5F092E02275F00280CB75F00480C675F00680C175F01680BC75F01780B7756C
:203E0E00F05780B2D2D575F05780AD75F01080A675F00880A175F001809C75F020809778CC
:203E2E00FB120043E6C0E008E6C0E0123DF913D0F0D0E0500224E02278FB120043E6C0E07F
:203E4E0008E6C0E0123DF413D0F0D0E050E924202278F712004386820886830886070808DF
:203E6E008603088604EB4C600AEFF0A31BBBFFF51C80F22278FB1200438682088683E4FBBC
:203E8E00FCFFE0A3B42D030FE0A3C39430B40A005012FA740A75F0001200B92AFBE5F034A3
:203EAE0000FC80E4EB8CF0DF0302013E2278F91200438682088683E0600DA380FA78F9121C
:203ECE0000438682088683088601088602C9C582C9CAC583CAE0A3C9C582C9CAC583CAF07C
:203EEE006003A380E8E5828583F02278FB1200438682088683E4F5F0FAE06009A30ABA0071
:203F0E00F805F080F4EA2278FB120043E60886F030F73A02013E78F9120043860308860477
:203F2E00088605088606ED8EF0120196401CED8EF02278F9120043860308860408860508D3
:203F4E008606ED8EF012019640E4EB8CF02278FB120043860308860485FEF0E5017F001239
:203F6E00017A600575F001E422EF0FF5F0A412017A70F6EF1475F0002278F9120043868215
:203F8E00088683088601088602C9C582C9CAC583CAE0F5F0A3C9C582C9CAC583CAE0B5F08C
:203FAE00056009A380E37401500274FF02008778F912004386820886830886F0E0B5F006D4
:203FCE008583F0E58222A370F3F5F022124121868208868308E4FEFFE07006124121E4F031
:203FEE0022B42551A3E0B42D05430780A3E0B4300343074024D0B40A00500BCE75F00AA452
:20400E002EFEA3E080EEE0B46413E60886F030F70843072012013EA6F018F68003B47505C7
:20402E0043070A8021B478054307108019B46F104307088011124121F0A3124121A3809510
:20404E00B462624307027A00C004C005C006C007AB0753031F7C00E60886F01200D3A6F07C
:20406E0018F6EDD007D006D005D0042430B43A0040022407C0E00AE645F070CC124121A914
:20408E0002EF30E505742DF0A30A12412AD0E0F0A3D9FA0808EF30E7A1EAC39E509C7420B4
:2040AE00F0A30A80F4B4630DAA0112412112412AE6F0A380DEB47331C082C08386820886D7
:2040CE00837A00E06004A30A80F9868318868212412112412A124121E0A31241216004F092
:2040EE00A380F2D005D00480AAB4691B86017A00E76004090A80F912412112412A8601E75B
:20410E006091F009A380F8F97A0112412112412AE9809ECDC583CDCCC582CC22EE601A8F46
:20412E00F020F715C002EAC39E500C742030F6027430F0A30A80EFD002220414170100401C
:20414E001454000000005445524D302000DE41436F6E736F6C652073746174757320666CB9
:20416E0061677320253032780A00205472616E733A20204865616420253032782C20546199
:20418E00696C20253032782C2043747220253032782C204D617820253032780A0020526517
:2041AE00633A202020204865616420253032782C205461696C20253032782C2043747220B9
:2041CE00253032782C204D617820253032780A003031323334353637383941424344454695
:2041EE00003030200020002A2A2A2042616420636865636B73756D3A202532780A002A009C
:20420E000A002A2120004F4B0A003E002A2A2A204E6F206164647265737320737472696E88
:20422E00672E2E2E0A004E657420616464726573732069732025730A004E6574206164641A
:20424E0072657373205B25735D002E2020537461636B207573656420253032782F25303219
:20426E00782E0A004572726F7220666C61677320253032782E20204E6574776F726B20634F
:20428E006865636B73756D206572726F72732025750A004C6F6767696E67206D6F646520F3
:2042AE0069732025750A004E6574206D6F64652069732025750A002A2A2A204E20636D6464
:2042CE002073796E746178206572726F720A002A2A2A20556E6B6E6F776E20636F6D6D61FA
:2042EE006E643A205B25735D0A002E2E2E203F3A000A002D2D2D20496E697469616C697AA9
:20430E00696E67204C43442E2E2E0020646F6E650A002D2D2D204C434420746F205B257572
:20432E002025755D2C20636D643D253032780A004C4344207363726F6C6C20757020257551
:20434E002E2E2E2020002E2E2E207363726F6C6C20646F6E650A004C43442025303278206A
:20436E005B25635D0A002020526561646261636B20636861727320617265205B005D0A002D
:20438E00202052656C6F6164656420636861727320617265205B00205D0A002D2D2D20413C
:2043AE004E534920636861722069732025303278205B25635D2C2073746174652025750A9B
:2043CE0000202020537461727420414E53492073657175656E63650A00202020204D6973EA
:2043EE0073696E67205B20636861722C2073657175656E63652063616E63656C6C65640A5B
:20440E00002020202042616420636861722025303278205B25635D2C2063616E63656C6CAC
:20442E0065640A002020202042616420636861722025303278205B25635D206166746572A5
:20444E0020706172616D2C2063616E63656C6C65640A0020202045787472616374696E67B3
:20446E0020706172616D2066726F6D205B25735D20402025753A2000284E756D2073747274
:20448E00696E67206973205B25735D292020002025750A0020202044756D70696E67207370
:2044AE00657175656E6365205B25735D0A002020205374617274206465636F64653A202022
:2044CE0000202020437572736F722075702025752000202020437572736F7220646F776E5B
:2044EE002025752000202020437572736F7220666F727761726420257520002020204375EF
:20450E0072736F72206261636B2025752000202020437572736F7220746F20414E534920F0
:20452E00726F772025752C20636F6C2025752000202020436C65617220616E6420686F6DF9
:20454E006520637572736F7200202020436C65617220746F20656E64206F66206C696E65CC
:20456E0000202020536574206C696E652077726170206D6F646500202020436C65617220D3
:20458E006C696E652077726170206D6F646500202020517565727920637572736F72206C06
:2045AE006F636174696F6E2028726F772025752C20636F6C20257529001B5B25753B257554
:2045CE00520A002020205361766520637572736F722028414E534920726F772025752C20D3
:2045EE00636F6C2025752900202020526573746F726520637572736F722028414E534920F7
:20460E00726F772025752C20636F6C2025752900202020496E76616C696420636F6D6D61B9
:20462E006E642063686172205B25635D202530327820686578000A001B000C000A000D00B0
:20464E0020002A2A2A204F75747075743A2020626164206269742049440A002A2A2A204F59
:20466E0075747075743A202062616420666F726D61740A00253032780A0045534554002A32
:20468E002A2A20556E6B6E6F776E20636F6D6D616E640A002A2A2A205320636F6D6D616E13
:2046AE006420737472696E67206973206D697373696E670A00417661696C61626C652063AD
:2046CE006F6D6D616E6473202876616C75657320696E20646563696D616C20756E6C6573D8
:2046EE0073206E6F7465640A0020413D737472696E6720202B2020736574206E6574776F7C
:20470E00726B206164647265737320746F20737472696E670A002044202020202020202080
:20472E00202A202064756D7020696E7465726E616C20737461747573207661726961626CE9
:20474E0065732028736F6D6520696E20686578290A0020452020202020202020202A2020F9
:20476E0073686F7720616E6420636C656172206572726F7220666C6167730A00204C206E75
:20478E002020202020202020202073657420646562756767696E67206F7574707574206D55
:2047AE006F64650A00204E206E2020202020202A2B2020736574206E6574776F726B206D55
:2047CE006F64650A00204F20783D6E2020202020202020736574206F7574707574206269CF
:2047EE0074207820746F207374617465206E0A0020512020202020202020202020207175EC
:20480E00657279206B65797320707265737365640A0020524553455420202020202020209B
:20482E00706572666F726D20706F7765722D6F6E20726573657420696E697469616C697AE8
:20484E006174696F6E0A0020533D737472202020202020202073686F7720737472696E67A4
:20486E00206F6E204C434420772F414E53492070726F63657373696E670A002B206D617257
:20488E006B73206E6574776F726B2D6F6E6C7920636F6D6D616E64730A002A206D61726BA2
:2048AE007320646562756767696E6720636F6D6D616E64730A000A4C43442D4C696E6B2077
:2048CE004E6574776F726B6564204C4344205465726D696E616C2C2056657273696F6E2076
:2048EE0000312E3061000A2020436F707972696768742031393932204369726375697420AF
:20490E0043656C6C61722C20496E632E0A004C43442D4C696E6B205625730A00312E306102
:20492E0000286329393220436972637569742043656C6C6172001B5B324A002D2D2D204605
:15494E00656C6C206F75742074686520626F74746F6D210A005E
:00000001FF
